:100000000C94E5050C941D060C941D060C941D061D
:100010000C941D060C941D060C941D060C941D06D4
:100020000C941D060C941D060C94DC2A0C94AE2B2B
:100030000C94B2240C941D060C941D060C941D0601
:100040000C941D060C941D060C941D060C941D06A4
:100050000C941D060C943B250C941D060C941D0657
:100060000C941D060C941D060C941D060C941D0684
:100070000C941D060C941D060C941D060C941D0674
:100080000C941D060C941D060C941D060C941D0664
:100090000C941D060C941D060C941D060C941D0654
:1000A0000C941D060C941D060C941D06790A790A01
:1000B000A50AA50A130B310B120C120C360B9E0B62
:1000C000AF0BAF0B4A1B4D1B771B8A1B921B9D1B53
:1000D000A01BA01BA01BE81BE81BA51BA81BAD1B9E
:1000E000BA1BC71BCA1BCE1BDB1B491CBB1C511CEC
:1000F0001B1C1F1C551C221C581C631C2D1CB11CD6
:10010000311C671C351C6B1C951C391C6F1C9F1CFB
:100110003F1C751C7F1C261C5C1C291C5F1C441C7E
:100120007A1C8B1CAB1CAD1C171C4D1CC41C322331
:10013000382326232C233E2344234A23162C3D2CEC
:10014000352D3D2C352D892CAC2C352D032D122D24
:10015000290014001A000800150017001C001800E0
:100160000C00120013004C002A004B002B0004006E
:100170001600070009000A000B000D000E000F001A
:100180003400280000004E00E1001D001B000600A6
:1001900019000500110010003600370038325200F7
:1001A00000003900E000E300E200215200000000FE
:1001B0002C000000E60022525000510000004F00C9
:1001C00001001E021F022002210222022302240239
:1001D00025022F003000310001004A0001001E00FE
:1001E0001F002000210022002300240025002600FB
:1001F0002700280000004D000100260227023300DE
:10020000370001002D002E02250238002E000100CB
:1002100000000100010001000100010000000000D9
:1002200001000000010001000100010000000100C8
:10023000A5003A003B003C003D003E003F000100AD
:10024000010001000100AC00AB00A900A6004000C5
:10025000410042004300440045000100010001004C
:100260000100AE000000AA00A7000100010001008B
:100270000100010001000100010001000100010076
:1002800000000100007C01000100010000000000EE
:100290000100000001000100010001000000010058
:1002A00044454255473A2064697361626C65642E27
:1002B0000A0044454255473A20656E61626C6564A8
:1002C0002E0A000A0025303258006C65645F7461A4
:1002D000736B3A20004F6E6573686F743A206163E8
:1002E000746976653A2025640A000A0025303136A3
:1002F00062003A200025303258000A722F63203005
:100300003132333435363738394142434445460A71
:1003100000290A002575002F002575005D2800259D
:10032000640020002564002000256400200025646E
:10033000007C0025303258006D6F7573656B6579F0
:10034000205B62746E7C782079207620685D28724C
:1003500065702F61636C293A205B0000000000008B
:100360000000002A2B280000000000000000000010
:1003700000000000000029000000002C1E34202195
:100380002224342627252E362D3738271E1F2021DC
:1003900022232425263333362E37381F040506073B
:1003A00008090A0B0C0D0E0F101112131415161755
:1003B00018191A1B1C1D2F3130232D350405060773
:1003C00008090A0B0C0D0E0F101112131415161735
:1003D00018191A1B1C1D2F3130354C00000000006D
:1003E000000000000000000000000000000000000D
:1003F0000000000000000000000000000000007E7F
:100400000F00D4FFFFFFC700000078313A09646590
:100410006C6179282A31306D73293A2025750A32AA
:100420003A09696E74657276616C286D73293A2099
:1004300025750A333A096D61785F73706565643AB2
:100440002025750A343A0974696D655F746F5F6DB4
:1004500061783A2025750A353A09776865656C5FD9
:100460006D61785F73706565643A2025750A363A68
:1004700009776865656C5F74696D655F746F5F6D42
:1004800061783A2025750A00703A097072696E74B5
:100490002076616C7565730A643A0973657420642B
:1004A000656661756C74730A75703A092B310A645C
:1004B0006E3A092D310A6C743A092B31300A727484
:1004C0003A092D31300A4553432F713A0971756944
:1004D000740A0A7370656564203D2064656C7461FC
:1004E000202A206D61785F7370656564202A20285A
:1004F000726570656174202F2074696D655F746F1B
:100500005F6D6178290A77686572652064656C742F
:10051000613A20637572736F723D25642C20776891
:1005200065656C3D25640A53656520687474703A8E
:100530002F2F656E2E77696B6970656469612E6F08
:1005400072672F77696B692F4D6F7573655F6B6588
:1005500079730A004D3E20004D25753A25733E20E3
:10056000003F0A003D2025750A003F0A00646566C9
:1005700061756C74730A0025750A003F0A000A0948
:100580002D2056616C756573202D0A00710A000AD2
:10059000092D204D6F7573656B6579202D0A003F1D
:1005A00000433E20004C25640A000A092D205374A4
:1005B00061747573202D0A686F73745F6B6579625F
:1005C0006F6172645F6C65647328293A202530324C
:1005D000580A6B6579626F6172645F70726F746FD5
:1005E000636F6C3A20253032580A6B6579626F610F
:1005F00072645F69646C653A20253032580A746908
:100600006D65725F72656164333228293A20253046
:10061000386C580A002573000A092D20436F6E7349
:100620006F6C65202D0A4553432F713A0971756926
:10063000740A6D3A096D6F7573656B65790A000A06
:10064000092D204D61676963202D0A443A094465EC
:10065000627567204D65737361676520546F6767C6
:100660006C650A583A094D61747269782044656274
:100670007567204D6F646520546F67676C65202D2A
:100680002053686F77206B6579707265737365733B
:1006900020696E206D617472697820677269640ADE
:1006A0004B3A094B6579626F6172642044656275EB
:1006B0006720546F67676C65202D2053686F772023
:1006C0006B65797072657373207265706F72740AEE
:1006D0004D3A094465627567204D6F757365205406
:1006E0006F67676C650A563A0956657273696F6E73
:1006F0000A533A095374617475730A433A094163A2
:1007000074697661746520436F6E736F6C65204DFC
:100710006F64650A46312D4631303A095377697462
:10072000636820746F204C6179657220302D392008
:1007300028463130203D204C30290A302D393A09E5
:1007400053776974636820746F204C6179657220F7
:10075000302D390A47524156453A09537769746337
:100760006820746F204C6179657220302028616C9C
:100770007465726E617465290A423A094A756D7032
:1007800020746F20426F6F746C6F616465720A45EC
:1007900053433A094A756D7020746F20426F6F742D
:1007A0006C6F616465722028616C7465726E61742F
:1007B00065290A453A095072696E742045455052C0
:1007C0004F4D2053657474696E67730A4241434B01
:1007D00053504143453A09436C6561722045455089
:1007E000524F4D0A006B65796D61705F636F6E6685
:1007F00069672E7261773A20253032580A2E737756
:1008000061705F636F6E74726F6C5F636170736C45
:100810006F636B3A2025750A2E636170736C6F638A
:100820006B5F746F5F636F6E74726F6C3A202575C7
:100830000A2E737761705F6C63746C5F6C677569A7
:100840003A2025750A2E737761705F7263746C5F4E
:10085000726775693A2025750A2E737761705F6C2F
:10086000616C745F6C6775693A2025750A2E737721
:1008700061705F72616C745F726775693A2025758B
:100880000A2E6E6F5F6775693A2025750A2E737799
:1008900061705F67726176655F6573633A20257585
:1008A0000A2E737761705F6261636B736C6173684A
:1008B0005F6261636B73706163653A2025750A2E10
:1008C0006E6B726F3A2025750A2E737761705F65C3
:1008D00073636170655F636170736C6F636B3A2003
:1008E00025750A0064656275675F636F6E66696788
:1008F0002E7261773A20253032580A2E656E616279
:100900006C653A2025750A2E6D61747269783A20FB
:1009100025750A2E6B6579626F6172643A202575C0
:100920000A2E6D6F7573653A2025750A006565633B
:100930006F6E6669673A0A64656661756C745F6CB0
:10094000617965723A2025750A003F000A6D6F755E
:1009500073653A206F66660A000A6D6F7573653AB3
:10096000206F6E0A000A6B6579626F6172643A20CB
:100970006F66660A000A6B6579626F6172643A207D
:100980006F6E0A000A6D61747269783A206F66664C
:100990000A000A6D61747269783A206F6E0A000A63
:1009A00064656275673A206F66660A000A6465626C
:1009B00075673A206F6E0A000A0A4A756D70696E93
:1009C0006720746F20626F6F746C6F616465722E44
:1009D0002E2E2000433E2000436C656172696E67D5
:1009E00020454550524F4D0A000A0025303258200C
:1009F000006B6579626F6172645F7265706F7274AB
:100A00003A20005B735D005B575D005B535D005BEC
:100A1000525D005B445D005B435D000C03340035B8
:100A20000041005400530000000E034100620065C5
:100A30000063003100330000000403090409027B55
:100A400000040100A0FA09040000010301010009EB
:100A5000211101000122400007058103080001095E
:100A600004010002030000000921110100012222FB
:100A70000007058203200001070503032000010988
:100A80000402000103000000092111010001227B82
:100A9000000705840320000109040300020300008D
:100AA0000009211101000122220007058503200011
:100AB00001070505032000011201000200000008E3
:100AC00013AB11450100010200010631FF0974A1B9
:100AD000010975150026FF00952075088102097629
:100AE000150026FF00952075089102C00660FF09D9
:100AF00061A1010962150026FF0095207508810299
:100B00000963150026FF00952075089102C00501B4
:100B10000902A10185020901A1000509190129089D
:100B2000150025019508750181020501093009317B
:100B30001581257F95027508810609381581257F65
:100B4000950175088106050C0A38021581257F95E7
:100B50000175088106C0C005010980A1018503193E
:100B6000012AB700150126B700950175108100C054
:100B7000050C0901A101850419012AA0021501260D
:100B8000A002950175108100C005010906A10105AB
:100B90000719E029E71500250195087501810295DF
:100BA00001750881010507190029FF150026FF00BE
:100BB0009506750881000508190129059505750137
:100BC0009102950175039101C00011241FBECFEF62
:100BD000DAE0DEBFCDBF04B603FE18C080918C03FF
:100BE00090918D03A0918E03B0918F038730904B2D
:100BF000A740B04B59F410928C0310928D031092C1
:100C00008E0310928F03E0E0F8E3099512E0A0E074
:100C1000B1E0E8E6FCE502C005900D92AC3BB107FF
:100C2000D9F723E0ACEBB2E001C01D92AC38B207BB
:100C3000E1F70E946A170C94322E0C940000FF9387
:100C4000EF93E091BC02F091BD02309709F0099555
:100C5000EF91FF910895FC018591803011F0EFDF55
:100C6000FBCF0895FF27E0E230E247FF0CC041953B
:100C700097FF09C0EDE26095709580959095611D94
:100C8000711D811D911D27FF02C0219530E350E2A7
:100C9000AA27660F771F881F991FAA1FA41710F095
:100CA000A41B63955A95A9F7AA3008F0A95FA05D27
:100CB000AF93F395611571058105910541F7ED320B
:100CC00011F4EF93F395F21718F43F93F395FBCFDC
:100CD0008F91B5DFFA95E1F70895E991F991859142
:100CE000803021F0853219F0AADFF9CF089520E095
:100CF000E89455915532C1F3503311F468945591ED
:100D00005A3348F4505390F3220F022E220F220F31
:100D1000200D250FF4CF0EF421958991999153362A
:100D200019F3533729F1533559F1BC018827992715
:100D3000E8945C3621F489919991689455915436E0
:100D400039F446EF7EF077FF0DC08FEF9FEF0AC0BA
:100D500055374AE039F0583540E121F0523642E04B
:100D600009F00895FF93EF937DDFEF91FF91B7CFE7
:100D7000FF93EF93FC0181918030B9F360DFFBCFEB
:100D8000FF93EF9368DFF1CFDF93CF93CDB7DEB75B
:100D90002596A3DFCF91DF910895CF93C82F60E010
:100DA0000E94120D882311F0589A01C0589861E0F2
:100DB0008C2F0E94120D882311F0599A01C0599866
:100DC00062E08C2F0E94120D882311F05A9A01C004
:100DD0005A988C2FCF91089583E008958330B0F412
:100DE0006430A0F44E3090F498E3899FF001112410
:100DF0008EE0689FE00DF11D1124E40FF11DEE0F50
:100E0000FF1FE05BFE4F85919491089580E090E094
:100E1000089581E0089581E008950E940B070895E8
:100E200008950E9410070895A5E0B0E0EAE1F7E018
:100E30000C949E2D49835A833091C30289819A81F3
:100E4000311114C0662359F0222349F00E94DB0DB2
:100E5000182F682F89819A810E94B70D03C00E94C4
:100E6000C90D182F69817A81812F04C00E94DB0D82
:100E700069817A810E94AC142596E3E00C94BA2D26
:100E8000FC01262F408151816281738184810E94FF
:100E90001407089581E00895CF93DF93EC0160E09B
:100EA0000E944007BE010E941107DF91CF91089573
:100EB000E1E0F0E0DF0102C0AA0FBB1F6A95E2F794
:100EC000BD01DF0102C0AA0FBB1F4A95E2F7AD01C9
:100ED000462B01C0EE0F2A95EAF7942F9823491369
:100EE00002C08E2B0895E0958E230895242F462F5F
:100EF000682F8091D9020E9458070E94090D089519
:100F00000E942E1608950E942816089508950E94A2
:100F1000950C0E9486072FEF84E39CE021508040CF
:100F20009040E1F700C0000008950E9487070E94EA
:100F3000612508950E9487070E94852508950F93D3
:100F40001F93CF93DF938C0161E00E944007EC0177
:100F5000B8010E94F01A882359F1B801CE010E940D
:100F60000D07882329F1B801CE010E941A23882396
:100F7000F9F0B801CE010E94F31B8823C9F0B80133
:100F8000CE010E948022882399F0F8018281882373
:100F9000F1F1C3308CE7D80781F160F4C130FCE790
:100FA000DF0769F1A8F4C115DC4789F50E949507B0
:100FB000C0E031C0CB35FCE7DF0739F1CC358CE739
:100FC000D80701F1CA35DC4711F50E9425121FC070
:100FD00080913903C82FC095C170C0FB80F9809300
:100FE0003903CC2329F082EB92E00E942B06E0CF5C
:100FF00080EA92E00E942B060EC00E942D120E94F1
:101000009A07D6CF0E941B1202C00E942912C80163
:101010000E940907C82F8C2FDF91CF911F910F914C
:1010200008950E948A240E94600808950E9464081E
:101030000E94932408958295982F937344E0949F7F
:10104000900111248C7C86958695282B822F85759E
:10105000880F2A7A2695822B0895CF93DF93D92F74
:101060000E941B08C82F8D2F0E941B082C2F30E0D8
:10107000322F2227A901482BCA01DF91CF91089571
:1010800008950E944008089581E008950895CF933F
:10109000DF93D82F0E944408C82F882319F08D2F82
:1010A0000E9446088C2FDF91CF9108950895CF9329
:1010B000C82F0E9441088C2F0E944708CF910895A5
:1010C00080E00E94570808950E9467230E945708F5
:1010D0000895CF930E946723C82F8091BE02C8173E
:1010E00089F1C093BE020E9420256093BF027093D5
:1010F000C0028093C1029093C2028091390382FFA3
:101100001EC080FF04C08AEC92E00E942B068091F2
:10111000390380FF0CC01F92CF9385EC92E09F9320
:101120008F930E94C4060F900F900F900F908091A4
:10113000390380FF04C083EC92E00E942B068C2FC1
:101140000E945708CF910895ABE0B0E0EAEAF8E0DA
:101150000C949F2D4F83588769877A878B876111FD
:101160000E944F119E012F5F3F4F86E0F9011192BF
:101170008A95E9F785E0FE013796D90101900D9235
:101180008A95E1F789819A814C815D81452B31F007
:101190009F3F31F491E08F3F19F403C091E001C00B
:1011A00090E090FF09C049815A816B817C818D81DB
:1011B0009E810E947B1005C0C9010E944A078111CF
:1011C000F2CF2B96E2E00C94BB2DFC018081918143
:1011D0000E94080E0895662319F00E94EF1702C0BE
:1011E0000E944A180E94C1180895CF93882309F4D9
:1011F000A9C0C82F8238C1F40E94672381FDA2C014
:1012000069E380910001909101010E944F240E94A6
:1012100073112FEF87EE93E0215080409040E1F76B
:1012200000C0000069E319C0833801F50E946723FC
:1012300080FD88C063E580910001909101010E94CA
:101240004F240E9473112FEF81EE94E021508040D3
:101250009040E1F700C0000063E5809100019091AB
:1012600001010E9452240E9473116CC08438C1F4A1
:101270000E94672382FD66C067E48091000190911F
:1012800001010E944F240E9473112FEF81EE94E020
:10129000215080409040E1F700C0000067E4DDCFBE
:1012A0008CEF8C0F813AF8F48C2F0E9485208111ED
:1012B00049C06C2F80910001909101010E94192476
:1012C000882349F06C2F80910001909101010E94C8
:1012D00052240E9473116C2F8091000190910101A2
:1012E0000E944F24C0CF80E28C0F883048F4C77032
:1012F00081E001C0880FCA95EAF70E943211B3CF8E
:10130000EBE5EC0FE33040F4F0E0EB5BFE4F808167
:1013100090E00E94C32316C0E8E5EC0FE93150F4D9
:10132000F0E0EE0FFF1FED5EFE4F808191810E9485
:10133000E82308C083E38C0F833120F461E08C2F15
:101340000E94EB08CF910895882309F468C0823881
:1013500079F40E94672381FF62C069E380910001F4
:10136000909101010E944F240E94731169E310C003
:101370008338B9F40E94672380FF51C063E58091F0
:101380000001909101010E944F240E94731163E5B6
:1013900080910001909101010E9452240E947311DA
:1013A0000895843879F40E94672382FF38C067E487
:1013B00080910001909101010E944F240E947311BD
:1013C00067E4E6CF9CEF980F913A10F4682FE0CFD6
:1013D00090E2980F983050F4877091E001C0990F17
:1013E0008A95EAF7892F0E943811D8CF9BE5980F8C
:1013F000933028F480E090E00E94C323089598E59C
:10140000980F993128F480E090E00E94E823089535
:1014100093E3980F933118F460E00E94EB0808956D
:101420001F93CF93DF93182FEB010E94F5082097AD
:1014300041F08FE99FE00197F1F700C0000021978C
:10144000F6CF812F0E94A409DF91CF911F910895BB
:10145000893319F060E070E002C060E570E00E943E
:10146000100A0895882321F00E9432110E947311FE
:101470000895882321F00E9438110E947311089565
:10148000A0E0B0E0E6E4FAE00C94992D7C01162F80
:10149000C72FFC01D281058102950F700E9428118F
:1014A0008823B9F0DD23A9F08C2F807F803421F0D0
:1014B00080E2810F883068F080916A0382FF09C062
:1014C00082E00E94D5110E94281191E0D82ED926E1
:1014D00001C0D12CCC2EC2948FE0C8228C2D90E07C
:1014E0008C30910508F09EC1FC01EA5AFF4F0C9424
:1014F000822D8C2F807FCF70882311F0C295C07F02
:10150000DD2399F0CC2309F479C180E2810F883082
:1015100010F0111104C08C2F0E94321103C08C2FC7
:101520000E9442110E94731169C1812F0E94A40977
:10153000CC2309F477C180E2810F883038F1112380
:1015400029F18C2F0E94481124C08C2F807FCF70EE
:10155000803211F0C295C07F112319F01130D1F102
:1015600043C080916A0382FD17C0DD2349F0CC237C
:1015700029F08C2F0E9432110E94731180E03FC12C
:1015800080E00E94A409CC2309F44CC18C2F0E9456
:1015900038110E94731146C1DD2371F0002341F020
:1015A000013031F40E9452118C2B0E945C113AC11F
:1015B0000E9452118C2B23C0011103C00E9469119B
:1015C0002EC0013009F42EC18C2F0E94390A0E94CE
:1015D000691128C1DD2321F0063008F023C10EC0B7
:1015E000053008F01FC11BC0DD2361F0002331F07E
:1015F000F701858180FF02C18F7085838C2F0E9447
:10160000320A10C1002359F0193309F008C1FFEF65
:1016100027EE83E0F15020408040E1F7FEC08C2FA0
:101620000E94390AFFC08C2F86958695837019F029
:10163000813061F0F7C0DD2321F0812F9C2F937062
:1016400002C080E090E00E94C323F4C0DD2321F0BB
:10165000812F9C2F937002C080E090E00E94E823CD
:10166000E9C06D2F812F0E94EB08E4C08C2F83709E
:1016700079F5D111DBC0412F429546954770440F53
:10168000440F212F2F70042E01C0220F0A94EAF775
:1016900014FF08C08FE090E001C0880F4A95EAF778
:1016A000809501C080E0C695C695C370822BC2307C
:1016B00049F058F4C13019F00E94FA0CB7C00E94EA
:1016C000F40CB4C00E94000DB1C00E94F10CAEC079
:1016D000DD2319F08C2F817001C08695882309F4D1
:1016E000A5C0412F429546954770440F440F212FC6
:1016F0002F70042E01C0220F0A94EAF714FF08C0CD
:101700008FE090E001C0880F4A95EAF7809501C00C
:1017100080E0C695C695C370822BC23049F058F45C
:10172000C13019F00E94550D81C00E944F0D7EC03E
:101730000E945B0D7BC00E94090D78C0CF70DD2335
:1017400039F08C2F0E942A0D812F0E94320A6EC020
:10175000812F0E94390A8C2F0E94360D67C0123FDC
:1017600021F128F4103F41F0113FC1F043C0133F75
:1017700019F1143F79F03EC0DD2341F0053008F047
:1017800051C08C2F8F710E94430D4CC0063008F061
:1017900049C0F7CF80916A0382FD18C0DD2339F07C
:1017A0008C2F8F710E942A0D3DC0DD23C9F38C2F31
:1017B0008F710E94360D36C0DD2329F08C2F8F717A
:1017C0000E94210D2FC00E940E0D2CC0DD2349F078
:1017D000CF718C2F0E942A0D63E08C2F0E94B711CD
:1017E00021C081E00E94D5110230E0F082E00E9429
:1017F000D51118C0DD2331F0002391F2812F0E9412
:10180000F50810C0002399F2193349F49FEFE7EE71
:10181000F3E09150E040F040E1F700C00000812F7C
:101820000E94A40988EF8C0D843020F40E94672365
:101830000E945708DD2089F00E94241180FD0DC010
:10184000F70112820E941E110E942A0DC7010E94F8
:101850004A0C0E941E110E94360DCDB7DEB7E8E09B
:101860000C94B52D0F931F93CF93DF93EC016881F8
:1018700079818A810E94130E8C010E94610D0E9461
:10188000E40CB801CE010E94400ADF91CF911F9174
:101890000F910895CF93DF93EC01988189812B817B
:1018A0003C81232B31F08F3F31F481E09F3F19F4CD
:1018B00003C081E001C080E080FD1AC0CE010E941B
:1018C0009F0781110FC00E942811882389F08A8107
:1018D000882371F080916A0382FF0AC082E00E942F
:1018E000D51106C0CE010E94320CCE010E944C07D9
:1018F000DF91CF91089580E090E00E94C32380E0C3
:1019000090E00E94E8230E944F110E9473110E94F0
:1019100062190E94C11808958091000190910101FF
:101920000E9455240E947B0C08950E943F110E9442
:101930008C0C089592959F70963079F010F4925027
:1019400001C09A50923068F4803F69F018F4883EE4
:1019500040F409C0843F29F406C0883E20F0813F4E
:1019600011F080E0089581E00895FC01908181816B
:1019700023813481232B31F08F3F31F481E09F3F6D
:1019800019F403C081E001C080E080FD07C08081C0
:1019900091810E94080E0E949A0C089580E008959B
:1019A000A5E0B0E0E6EDFCE00C949F2D2596E2E08A
:1019B0000C94BB2DA6E0B0E0E0EEFCE00C949F2D73
:1019C0002696E2E00C94BB2D089508950E94E50C44
:1019D00008950E94E60C08950E94E90C8093DA02B3
:1019E00008950E94EC0C08959091DA02892B0E94D0
:1019F000EC0C08959091DA0289230E94EC0C089572
:101A00009091DA0289270E94EC0C08950E94CD067D
:101A100008950E94060D8093D902089580E00E94E7
:101A2000090D0895811105C081E0662349F080E029
:101A3000089590E002C0959587956A95E2F78170C8
:101A4000089591E001C0990F8A95EAF7892F0E94C5
:101A5000090D089521E030E001C0220F8A95EAF7D0
:101A60008091D902822B0E94090D089521E030E077
:101A700001C0220F8A95EAF720958091D90282232E
:101A80000E94090D089521E030E001C0220F8A95DF
:101A9000EAF78091D90282270E94090D089590915A
:101AA000D902892B0E94090D08959091D9028923AA
:101AB0000E94090D08959091D90289270E94090D6D
:101AC00008950895962F9770A1E001C0AA0F9A95E6
:101AD000EAF793E0769567959A95E1F7FB01EE0FAB
:101AE000FF1F6E0F7F1FFA01E60FF71F40E050E067
:101AF000682F70E090819B01042E02C036952795D7
:101B00000A94E2F72170219529272A232927219376
:101B10004F5F5F4F4330510569F708959B01782F60
:101B2000777043E0969587954A95E1F7FC01EE0FB3
:101B3000FF1F8E0F9F1FF901E80FF91F40E050E0D3
:101B400080E0219130E0072E02C0369527950A9457
:101B5000E2F721703327042E01C0220F0A94EAF71E
:101B6000822B4F5F5F4F4330510559F70895282F5F
:101B7000943070F48E3060F4862F622F70E02EE087
:101B8000929F600D711D112444EC52E00E94620D81
:101B90000895943070F48E3060F4292F90E064EC56
:101BA00072E03EE0239F800D911D11240E948E0D56
:101BB000089580E00895CF92DF92FF920F931F93D4
:101BC000CF93DF936C010091D9028091DA02082B48
:101BD000C7E0D0E010E0C8010C2E02C095958795B3
:101BE0000A94E2F780FD04C02197A8F7F12C07C002
:101BF000FC2EB6018C2F0E94B8140197A9F38F2DEB
:101C0000DF91CF911F910F91FF90DF90CF900895BA
:101C1000CF93DF93EC010E94DB0DBE010E94B8144C
:101C2000DF91CF9108951F93CF93DF93EB019091B4
:101C3000C302992321F0CB010E94080E13C0882310
:101C400049F0CB010E94DB0D182F682FCE010E94B6
:101C5000B70D04C0CB010E94C90D182FBE01812F02
:101C60000E94B814DF91CF911F9108951F93CF93D5
:101C7000DF93C091DB0216E08091DC02C81799F077
:101C8000D0E01C9FF0011D9FF00D1124E352FD4F89
:101C90004081518162817381848195810E94DA0C37
:101CA0002196C770E9CFDF91CF911F9108954091A0
:101CB0000D0350910E0360910F03709110038091FA
:101CC0001103909112030E94DA0C08950F931F9351
:101CD000CF93DF938091120382958F7009F05AC0E1
:101CE00080910F03882309F455C08091DB02109185
:101CF000DC0260910D0370910E03C0911003D0912E
:101D0000110391E06F3F09F090E0292F06E0811761
:101D100009F440C0209721F07F3F21F030E003C05C
:101D200031E001C0322F90E030FD31C0089FF0015A
:101D3000099FF00D1124DF01A352BD4F11963C9174
:101D40001197371324C03C91361321C012963C9151
:101D5000129731111CC013964D915C9114974C1B36
:101D60005D0B483C510598F4809112038F7080619F
:101D700080931203EE51FD4F80818F7080618083CC
:101D80008DE093E00E944A0C0E94360E03C001963B
:101D90008770BDCFDF91CF911F910F910895A1E181
:101DA000B0E0E5EDFEE00C94962D8C0185E0F801A5
:101DB000DE011D9601900D928A95E1F7F801E2800F
:101DC00090910D0360910E03209110033091110347
:101DD0002115310531F06F3F31F481E09F3F19F457
:101DE00003C081E001C080E0F82FF1709F2E80FDDC
:101DF00040C1F80140815181A380B4808DE0C82E9C
:101E000083E0D82EF0900F03F501E21BF30BFF20C7
:101E100009F4DAC080911203E83CF10508F096C09D
:101E2000282F207F09F053C0561313C0491311C047
:101E3000FE2CE1100EC08F708061809312030E940F
:101E4000570EC6010E944A0C80911203F801858347
:101E50004DC1A114B10431F05F3F31F481E04F3F37
:101E600019F403C081E001C080E080FD03C081E07F
:101E70008E2502C080E090E0F82FF170FF2E80FFE9
:101E80001CC08091DB022091DC0236E0821709F44D
:101E90000BC190E0389FF001399FF00D1124E352FF
:101EA000FD4F6181561306C06081461303C06281F5
:101EB000E61203C001968770E9CFFE2CEE2009F4EC
:101EC00015C18091120381608093120354C0561390
:101ED00006C0491304C0E11002C0F80199C0C8014E
:101EE0000E94B50C882361F1EE2051F1209112037C
:101EF000822F82958F7090E0029774F080910D038D
:101F000090910E0398878F831986BB86AA862C87AB
:101F1000CE0107960E944A0C86E0F801ADE0B3E0DE
:101F200001900D928A95E1F70E94660E0E94570E6D
:101F30000AC0561711F1C8010E94B50C81112CC0BE
:101F4000C8010E944A0CFF24F394D0C0282F207FA0
:101F500081F77A2DB98AA88A6E2D89890E94D00CC2
:101F60008DE093E00E944A0C86E0F60111928A957A
:101F7000E9F70E94570EF12CB9C04913DCCFE110EC
:101F8000DACFF8018583C8010E944A0C86E0F60189
:101F900011928A95E9F7AAC0EE2091F220911203DE
:101FA000822F82958F7090E002970CF4B5CF8091CC
:101FB0000D0390910E039A8389831B82BD82AC82AC
:101FC0002E83CE010196A6CFE83CF10508F044C06F
:101FD000FE2CEE2009F4B4CF561330C049132EC0A6
:101FE0002091120320FD21C0822F82958F70482FEF
:101FF00050E041155105C9F0F80125834F305105D6
:1020000041F08F5F982F9295907F822F8F70892B50
:102010008583C8010E944A0C86E0F801ADE0B3E078
:1020200001900D928A95E1F73CC086E0F801ADE0A1
:10203000B3E001900D928A95E1F758C0C8010E9463
:10204000B50C811169CF80911203816080931203D6
:10205000C8010E944A0C4AC07A2DB98AA88A6E2DFE
:1020600089890E94D00C86E0F60111928A95E9F7E1
:1020700018C0EE2009F464CFC8010E94B50CF82EF8
:10208000882309F45DCF86E0F801ADE0B3E001906C
:102090000D928A95E1F78DE093E00E94E5080E9499
:1020A000660E0E94570E22C04D875E878D859E85E5
:1020B0000E94080E292F22952F70223028F49F703D
:1020C00039F0811105C00BC0243028F49F7049F409
:1020D000805E883020F0C8010E944A0C9F2CF92CA9
:1020E00005C0F8019581907F99F7F9CF8F2D619602
:1020F000EBE00C94B22DACE0B0E0E1E8F0E10C9440
:102100009E2D4F83588769877A878B879C87CE015E
:1021100007960E94CF0E8823D1F09F8188852A855B
:102120003B85232B31F08F3F31F481E09F3F19F441
:1021300003C081E001C080E080FD47C04F81588529
:1021400069857A858B859C850E94DA0C3EC086E085
:10215000FE013796DE01119601900D928A95E1F706
:10216000FF81E8856A857B856115710531F0EF3F58
:1021700031F481E0FF3F19F403C081E001C080E049
:1021800080FD23C02091DC0230E0C90101968770F8
:1021900099274091DB0250E084179507F1F1F9830C
:1021A000EA837D836C8396E0929FD001939FB00D6C
:1021B0001124A352BD4FFE01319601900D929A95C4
:1021C000E1F78093DC020E94360E16E08091DB027C
:1021D0009091DC02891771F1189FC001112483527C
:1021E0009D4F0E94CF0E882329F1E091DB021E9FB4
:1021F000F0011124E352FD4F4081518162817381CE
:10220000848195810E94DA0C8091DB0290E0019636
:10221000877099278093DB02D9CF0E94950C10928A
:10222000DC021092DB02EDE0F3E086E0DF011D92BC
:102230008A95E9F72C96E3E00C94BA2D80911B0364
:10224000859585958595089580911B0387700895E0
:1022500090911B03977081E009F480E008958091CC
:102260002603089590912603892B809326030895D1
:1022700080959091260389238093260308951092D8
:102280002603089590912503892B809325030895B3
:1022900080959091250389238093250308951092BA
:1022A0002503089580911C03089508950E945511F7
:1022B00008950E945611089590916A0392FF08C0F4
:1022C00090911C03981721F080931C030E945911D0
:1022D000089580911C03882329F010921C0380E04C
:1022E0000E9459110895CF93DF93E0910001F0917E
:1022F0000101809126038083E0910001F0910101AA
:10230000908180912503892B808380911C038823F1
:1023100081F0E0910001F09101019081892B80838F
:1023200080910001909101010E940D2481110E9471
:102330006911C0910001D091010148E050E063E1D2
:1023400073E0CE010E94DA2D892B59F088E0FE015E
:10235000A3E1B3E001900D928A95E1F7CE010E94CE
:102360007423DF91CF9108950E94551108959091A3
:102370006A0392FF11C098E0899F90011124262BD7
:1023800020931B030E942A0D80911B038595859540
:1023900085950E94B41108950E942A0D0895109207
:1023A0001B0380E00E94B411089520911B038095C7
:1023B000822380931B03982F977099F430E0482F65
:1023C000082E000C550B2417350759F090916A031D
:1023D00092FF07C08595859585950E94360D0E94D0
:1023E000CF110895CF9390916A0392FB222720F991
:1023F0002817F9F0C82F892FC0FB82F980936A0350
:102400008091690390916A030E944F1282E00E94BA
:10241000D5118091390380FF0CC01F92CF9385EDB9
:1024200092E09F938F930E94C4060F900F900F909D
:102430000F90CF91089580916A0382FB882780F9DD
:1024400091E089270E94F211089581E00E94F21123
:10245000089580E00E94F21108956FEF7FEF80E011
:1024600090E00E941C2E089580E090E00E94F82DDC
:10247000873E9E4F19F40E94841A089580E00895C3
:1024800082E090E00E94F02D089583E090E00E94A9
:10249000F02D089584E090E00E94F82D0895BC018D
:1024A00084E090E00E941C2E0895AB01BC018FE0F7
:1024B00090E00E94102E0895AB01BC0183E190E0F2
:1024C0000E94102E089560E070E0CB010E945C1223
:1024D000089560E070E0CB010E9455120E946312E3
:1024E000089567EE7EEF80E090E00E941C2E60E091
:1024F00082E090E00E94FE2D60E083E090E00E9488
:10250000FE2D1092DA0260E074E184E090E00E9417
:102510001C2E60E086E090E00E94FE2D6FEF87E0C9
:1025200090E00E94FE2D40E050E0BA0188E090E08B
:102530000E94102E60E08DE090E00E94FE2D40E0B1
:1025400050E0BA0188E190E00E94102E60E087E13F
:1025500090E00E94FE2D40E050E0BA018CE190E056
:102560000E94102E60E070E080E290E00E941C2E3D
:1025700040E050E0BA0188E190E00E94102E80E037
:102580000E949D1A0E94D21A0E94691208950E9408
:1025900071120895682F8EE090E00E94FE2D08953C
:1025A0000E94202560933503709336038093370390
:1025B0009093380360933103709332038093330315
:1025C00090933403089581E008950E94E3120895E2
:1025D00008950E94E81208950E94E81208950E944A
:1025E000EC1208950E94E81208950E94F2120895D4
:1025F0000E94E812089584E497E20E945D230E94FD
:10260000F8120E94F51208950E94E9120E94E81241
:1026100008950E94B6150E94560808950E940B2541
:102620000E94E21A0E94CF160E9409130E94EF1224
:102630000895AAE0B0E0EFE1F3E10C94942D0E943C
:10264000E51629E2E22E23E0F22E5701D12CF50106
:10265000019111915F018D2D0E94D1158027912745
:10266000D394F4E0DF1619F0892B89F322C0892B6B
:1026700001F50E9414258C01809127039091280375
:102680000817190709F45BC08FEF89838A831B82BF
:102690000E9414258160782F9D838C8349815A8103
:1026A0006B818D810E94A408109328030093270357
:1026B00046C08091390381FD0E94DA150E94E5121F
:1026C000782E10E0812F0E94D1154C01F701A080D7
:1026D000B180A826B926A114B10449F100E0CC24A8
:1026E000C394D12CC5018C219D21892BC1F0772069
:1026F000B1F00E831F8321E0C4018C219D21892B21
:1027000009F420E028870E9414258160782F9A8799
:1027100089874E815F8168858A850E94A4080F5F42
:10272000CC0CDD1C0E30F1F6F701918280821F5F28
:10273000F2E0EF0EF11C143029F60E94D0120E9434
:1027400084190E9469082A96EDE00C94B02DCF936D
:10275000DF930E94BD14EC01811520E59207E0F59E
:10276000811530E4930708F09FC0803E910528F55D
:102770008D3C910508F096C0883A910570F4853A31
:10278000910508F085C08130910509F47EC008F4F8
:10279000DCC0049708F0DCC0D8C0813C910508F08B
:1027A000D4C0C85AD0E0CC0FDD1FC85BDE4F099003
:1027B000D881C02DCE019464CCC0811540E294072D
:1027C00008F0B8C0811551E0950708F0C1C0883EF7
:1027D000910508F4BDC0B9C0803662E5960720F5C2
:1027E000803472E5970708F06CC0C03282E5D807E4
:1027F00008F05EC0C11592E5D90708F489C02C2FF6
:102800002695269560E2269F90011124C37081E0F1
:1028100090E002C0880F991FCA95E2F7E901C82B22
:10282000D92BCE019D6895C0803A22E59207E0F44D
:102830008F71C03832E5D30708F059C08695869568
:1028400070E2879F900111249C2F9370C1E0D0E02B
:10285000AE0102C0440F551F9A95E2F7EA01DA680B
:10286000C9018C2B9D2B75C0803C42E5940708F470
:1028700045C0803E924508F068C0CF71DD27DC2F4F
:10288000CC27CE01806F906A64C081E090E061C087
:10289000C55AD0E0C658DE4F8881C82FD0E0CE019F
:1028A000906457C0906555C0DF70CE01906A51C0EA
:1028B000CF718C2F90E0D82FCC27CE01816F906AFA
:1028C00048C08F718695869570E2879FA00111247C
:1028D0009C2F937021E030E0B90102C0660F771F92
:1028E0009A95E2F7CB019C68842B952B32C090E03F
:1028F000D82FCC27CE01846F906A2BC08F710E9495
:1029000059158F7190E0D82FCC27CE01906221C04D
:102910008C2F8F710E94591595E0D695C7959A9581
:10292000E1F7CF70D0E0DC2FCC27D069BE01682B57
:10293000CB010FC08D2F8F710E945915DD27D062FA
:102940008F719E01382BC90104C080E090E001C066
:10295000CE01DF91CF910895743038F46E3028F4B1
:10296000462F672F0E949821089580E090E00895F7
:102970000E94AC140E94A71308958238910569F152
:10298000B0F48133910509F475C048F4893291059A
:1029900009F467C08A32910509F471C0089585333E
:1029A000910509F459C089339105B9F00895833E22
:1029B000910589F138F4803E9105D1F0823E910570
:1029C00029F10895863E9105C9F1873E9105D9F117
:1029D000843E910509F06CC027C02091690320FD59
:1029E00057C021FD55C020916A0323FD5BC00895A7
:1029F0008091690380FD48C080916A0380FF48C0D0
:102A00008091690384FD46C083EE51C080916903C3
:102A100082FF3CC0F5CF8091690382FD37C0809171
:102A20006A0380FD35C0ECCF80916A0381FF36C018
:102A30008091690384FD2EC087EE39C080916903BF
:102A400083FF2AC0F5CF8091690383FD25C0809163
:102A50006A0381FD23C0ECCF8091690385FD22C00C
:102A60001FC08091690385FD1BC080916A0383FFAD
:102A700019C00AC08091690386FD16C017C08091F5
:102A8000690386FD13C010C089E311C082EE0FC038
:102A900080EE0DC080E00BC086EE09C084EE07C05A
:102AA00085E305C089E203C08AE201C081E390E0CA
:102AB00008959091690392FF0DC0282F2871283046
:102AC00019F4877F846006C0282F2471243011F404
:102AD0008B7F886093FF0DC0282F2871283119F44F
:102AE000877E846106C0282F2471243111F48B7EE7
:102AF000886120916A0320FF0DC0382F387138306B
:102B000019F4877F816006C0382F3171313011F49C
:102B10008E7F886021FF0DC0282F2871283119F47D
:102B2000877E816106C0282F2171213111F48E7EAC
:102B3000886194FD877E08950E942D1208950E9459
:102B4000E5168FE39CE90197F1F700C000000E94B1
:102B5000E51680E00E94D11580FF04C00E949C15FC
:102B60000E94612508950E949F1508950E943412C5
:102B7000811102C00E94C7120E9440128093390343
:102B80000E944A1290936A03809369030E94B315CE
:102B90000E9445120E94F10C8091D9020E94060DFC
:102BA0000895E82FF0E0EE0FFF1FED58FC4F8081F5
:102BB00091810895A0E0B0E0E0EEF5E10C94992D4C
:102BC0008AEF92E00E942B0683E7E82E83E0F82E3E
:102BD000C0E0D0E095EFC92E92E0D92E0CEE12E0C5
:102BE000DF93CF93DF92CF920E94C40682EF92E0F0
:102BF0000E942B06F701819191917F010E942D087F
:102C00009F938F931F930F930E94C4068AEE92E0C6
:102C10000E942B0621968DB79EB708960FB6F894A2
:102C20009EBF0FBE8DBFC430D105D1F6CDB7DEB784
:102C3000E8E00C94B52D80EA8A95F1F7089500C07C
:102C400008950E941B16089508950E942416089561
:102C50000E94251608950E94241608950E942B169E
:102C60000895F894E82FE295EF70F0E031A1282F55
:102C70002F7081E090E001C0880F2A95EAF7982F25
:102C80009095932391A392A1892B82A37894089580
:102C90000F931F93CF93DF93CBE8D1E089918F3FC0
:102CA00011F00E94311681E0CF38D807B9F7CDE78F
:102CB000D1E00BE811E089918F3F11F00E943116AD
:102CC0000C171D07C1F7DF91CF911F910F91089548
:102CD000A0E0B0E0EEE6F6E10C94982D8C01C62F52
:102CE000D0E0CE0185579E4F6C01FC0190819F3F43
:102CF00009F450C0B62EF894E92FE295EF70F0E099
:102D000081A19F7021E030E001C0220F9A95EAF77F
:102D1000822B81A382A12095282322A378940E944C
:102D20001F16EDE7F1E04BE851E021E030E0E12C47
:102D3000F12C61916F3F89F0A62FA295AF70B0E0A2
:102D400090968C9190E06F7002C0959587956A95EA
:102D5000E2F780FD02C0C90102C080E090E0E82AED
:102D6000F92A220F331F4E175F0719F7F6018081EA
:102D70008F3F11F00E94311661E0E114F10409F473
:102D800060E08B2D0E942116CC0FDD1FC00FD11FDC
:102D9000F982E882CDB7DEB7E9E00C94B42D0E9449
:102DA000481688E0E3E7F3E0DF01982F1D929A953B
:102DB000E9F7EBE6F3E0DF011D928A95E9F784E09D
:102DC0000E9420170E9480070895A8E0B0E0EBEE73
:102DD000F6E10C949C2D8E010F5F1F4F88E0F801E7
:102DE00011928A95E9F7F12C6F2DC8010E9468169F
:102DF000F394F4E0FF12F8CF48E050E0B8018BE61E
:102E000093E00E94DA2D21E0009709F420E0892B5D
:102E100041F088E0F801ABE6B3E001900D928A95AD
:102E2000E1F744E063E773E08BE693E00E9421174B
:102E3000182F0E948307812F2896E5E00C94B82D67
:102E40000895EF92FF920F931F93CF93DF937C012E
:102E50008B01C42F222349F081E080933C030E9420
:102E6000142590933B0380933A0380913C03811196
:102E700002C080E01CC080913A0390913B030E9405
:102E80002C250597B0F3D0E0CC0FDD1FAE01B701C4
:102E9000C8010E94DA2D892B39F0AE01B701C801B3
:102EA0000E94E72D81E001C080E010923C03CDB785
:102EB000DEB7E6E00C94B72D0E94C1270E940E13E6
:102EC0000E94CE2708950E94D3270E9419130E94C2
:102ED000F12708950E94AB240E94A7270E94FB12AD
:102EE0000E945C170E9463170E940413FBCF80911D
:102EF000430380FF06C06091070170E0660F771FF3
:102F000026C081FF04C06091070184E005C082FFF4
:102F100007C06091070188E0689FB001112417C0C5
:102F2000909142039923D1F060910601961788F79A
:102F30002091070188E0289F90011124929FA00111
:102F4000939F500D112470E0CA010E946E2D6038CD
:102F5000710540F46115710519F406C068E070E070
:102F6000862F08958FE7089581E0089580914303A7
:102F700080FF08C06091030170E0759567957595B5
:102F8000679521C081FF06C06091030170E07595CF
:102F9000679519C082FF04C06091030170E010C002
:102FA00090914103992399F0609102019617A0F73F
:102FB00080910301899FC001112470E00E946E2D51
:102FC0006038710540F46115710519F406C061E0BF
:102FD00070E0862F08958FE7089581E008958D3C75
:102FE00021F40E947717819504C08E3C29F40E9439
:102FF00077178093470308958F3C21F40E94771739
:10300000819504C0803D29F40E9477178093460380
:103010000895893D19F40E94B61705C08A3D31F420
:103020000E94B61781958093480308958B3D21F443
:103030000E94B617819504C08C3D29F40E94B617F2
:103040008093490308959FE2980F983078F421E027
:1030500030E0A90102C0440F551F9A95E2F7CA015A
:1030600090914503892B8093450308958D3D21F46C
:103070008091430381600BC08E3D21F48091430316
:10308000826005C08F3D29F4809143038460809362
:10309000430308958D3C39F49091470397FF35C061
:1030A0001092470359C08E3C29F49091470319169A
:1030B000BCF32BC0909146038F3C29F497FF25C0A9
:1030C0001092460349C0803D19F41916CCF31DC077
:1030D00090914803893D29F41916BCF410924803D5
:1030E0003BC08A3D19F497FF10C0F8CF8B3D39F4EF
:1030F0009091490397FF09C0109249032DC08C3D60
:1031000021F4909149031916BCF39FE2980F98306F
:1031100080F421E030E0A90102C0440F551F9A95C8
:10312000E2F7CA0180959091450389238093450376
:1031300013C08D3D21F4809143038E7F0BC08E3DE3
:1031400021F4809143038D7F05C08F3D29F4809148
:1031500043038B7F8093430380914603811106C014
:1031600080914703811102C010924203809148036D
:10317000811106C080914903811102C01092410360
:1031800008958091390383FF7EC088E393E00E9415
:103190002B06809145031F928F9383E393E09F93C7
:1031A0008F930E94C40681E393E00E942B068091D6
:1031B0004603282F082E000C330B3F938F938EE28B
:1031C00093E09F938F930E94C4068CE293E00E9449
:1031D0002B0680914703282F082E000C330B3F93BA
:1031E0008F9389E293E09F938F930E94C40687E2B6
:1031F00093E00E942B0680914803282F082E000C94
:10320000330B3F938F9384E293E09F938F930E94BD
:10321000C40682E293E00E942B0680914903282F86
:10322000082E000C330B3F938F938FE193E09F9315
:103230008F930E94C4068CE193E00E942B0680913C
:1032400042031F928F9389E193E09F938F930E9493
:10325000C40687E193E00E942B06809143031F92EE
:103260008F9384E193E09F938F930E94C40681E142
:1032700093E00E942B068DB79EB74C960FB6F8943C
:103280009EBF0FBE8DBF0E941425209146032111C1
:1032900004C020914703222321F0909340038093A0
:1032A0003F0320914803211104C0209149032223A8
:1032B00021F090933E0380933D0384E493E00E94C9
:1032C000B5230895E4E4F3E086E0DF011D928A95DA
:1032D000E9F71092420310924103109243030895BC
:1032E000FC01828181110DC0838181110AC084811A
:1032F000811107C091E08581811101C090E0892F83
:1033000001C081E081700895A6E0B0E0EAE8F9E14B
:103310000C949E2D86E0E4E4F3E0DE01119601902A
:103320000D928A95E1F7109246031092470310928E
:103330004803109249038B81811104C08C8188233A
:1033400009F45FC080913F03909140030E942C25B7
:10335000AC0190914203992339F02091080130E0AB
:103360002417350758F04DC0209109018AE0289FA5
:10337000900111242417350718F043C09F3F19F01E
:103380009F5F909342031B81112361F00E94771786
:10339000111614F09FEF01C091E0989F902D112419
:1033A000909346031C81112361F00E947717111638
:1033B00014F09FEF01C091E0989F902D11249093FD
:1033C0004703309146033323E1F020914703222342
:1033D000C1F045EB3403C0011124992319F09093F7
:1033E000460303C081E08093460335EB2303C0010D
:1033F0001124992319F09093470303C081E080932F
:1034000047038D81811104C08E81882309F45FC038
:1034100080913D0390913E030E942C25AC01909138
:103420004103992339F02091040130E02417350736
:1034300058F04DC0209105018AE0289F9001112489
:103440002417350718F043C09F3F19F09F5F9093F2
:1034500041031D81112361F00E94B617111614F06B
:103460009FEF01C091E0989F902D11249093480305
:103470001E81112361F00E94B617111614F09FEF00
:1034800001C091E0989F902D1124909349033091B1
:1034900048033323E1F0209149032223C1F045EB97
:1034A0003403C0011124992319F09093480303C0F9
:1034B00081E08093480335EB2303C0011124992355
:1034C00019F09093490303C081E080934903BE0142
:1034D0006F5F7F4F84E493E00E945C24811105C0FC
:1034E00084E493E00E94701981110E94C11886E063
:1034F000FE013196A4E4B3E001900D928A95E1F7C4
:103500002696E3E00C94BA2D82E290E00E94F02D22
:10351000823281F483E290E00E94F02D823151F4F6
:1035200084E290E00E94F02D91E0883009F090E074
:10353000892F01C080E081700895CF93C82F811139
:1035400002C06FEF01C062E282E290E00E94FE2DB5
:10355000C11102C06FEF01C062E183E290E00E94FE
:10356000FE2DC11102C06FEF01C068E084E290E05F
:103570000E94FE2DCF910895089585E290E00E946B
:10358000F02D682F70E080E090E008950895CF93CB
:10359000C62F0E94C61A6C2F85E290E00E94FE2D75
:1035A000CF91089580E00E949D1A60E070E0CB0109
:1035B0000E94C71A0E942B210E94ED2181E00E94E7
:1035C0009D1A08950E94BC1A0E94BD1A0E94C61A34
:1035D0000E94841A811102C00E94D21A089508958F
:1035E000CF93FB01C281CC23E9F09C0122503747E5
:1035F0002031310520F482500E94FD210CC081153C
:10360000F7E79F0751F481E00E942A0D43E062E052
:1036100081E00E947607C0E018C081309747A9F486
:1036200082E0F2CF8115E7E79E0711F481E004C044
:103630008130974749F482E00E94360D43E062E012
:1036400081E00E94760701C0C1E08C2FCF910895E0
:103650002FEFFC01208308950E94281B089580E02D
:103660000895EF92FF920F931F93CF93DF93EC0196
:10367000062F0E942F1B8111B1C0E8818E2F90E090
:10368000FC013197E331F10508F0A2C0EE59FF4F7C
:103690000C94822D19828BE05EC08981823089F082
:1036A00030F4813009F094C00E9420250CC0833092
:1036B00079F0843009F08CC01A821B821C821D8232
:1036C00089C00E94BD1A9A838B837C836D8382C0DC
:1036D0007E0110E0812F0E94D115F7019283838330
:1036E0001F5FF2E0EF0EF11C1430A1F773C0898167
:1036F000823039F0853009F06BC08A810E94EF1A60
:1037000069C06A817B818C819D810E94882D0E9485
:10371000C71A60C04B816A8189810E94EF209C8317
:103720008D8358C02C813D813227232732274B813E
:103730006A8189810E9410214DC00E942B214AC0BC
:10374000602FCE010E942C1B45C00E94A42124C0E2
:103750000E94A62199838A833DC06B8170E0898194
:103760009A81AE014C5F5F4F9827892798270E9466
:10377000A92130C06B8170E089819A81AE014C5FD4
:103780005F4F9827892798270E94CC2123C00E9449
:10379000ED2120C00E94DC2089831CC06B8170E079
:1037A00089819A81AE014C5F5F4F982789279827BE
:1037B0000E9456210FC06B8170E089819A81AE0111
:1037C0004C5F5F4F9827892798270E94782102C075
:1037D0008FEF8883602FCE010E94D925CDB7DEB749
:1037E000E6E00C94B72DCF93DF93FC01DB0112963A
:1037F0008C91882309F4DDC09F01305723323105B5
:1038000008F0D8C0EF010E944A1290936A03809397
:103810006903FE01E150F047E232F10520F4EB5874
:10382000FF4F0C94822D809169038160AAC0809122
:103830006A038860B2C0809169038260A2C08091EF
:10384000690320C08091690388609BC080916A03EE
:103850001EC080916A038260A0C08091690380616C
:1038600090C08091690380628CC0809169038064FC
:1038700088C00E94950C80916903806882C0809105
:103880006903886084607DC080916A038260816082
:1038900084C0809169038E7F74C080916A03877FA2
:1038A0007CC0809169038D7F6CC08091690320C0CA
:1038B00080916903877F65C080916A031EC08091F3
:1038C0006A038D7F6AC0809169038F7E5AC08091A0
:1038D00069038F7D56C0809169038F7B52C00E941F
:1038E000950C809169038F774CC080916903877F25
:1038F0008B7F47C080916A038D7F8E7F4EC0809101
:10390000690382FB222720F991E0922790FB82F93C
:1039100090FB83F936C080916A03982F909591703F
:103920008E7F892B90FB81F938C08091690386FBDB
:10393000222720F991E0922790FB86F922C00E946D
:10394000950C8091690387FB222720F991E092274B
:1039500090FB87F916C081E001C080E00E94CA1286
:103960001EC08091690384FB222720F991E09227F1
:1039700090FB84F906C080916903982F909590FB85
:1039800080F9809369030BC080916A0383FB22272F
:1039900020F991E0922790FB83F980936A0380914C
:1039A000690390916A030E944F120E94950C80E077
:1039B00001C081E0DF91CF910895A0E0B0E0E3EE97
:1039C000FCE10C949A2DE82FF0E0E55AFC4FD490DE
:1039D000282F26952695269530E0F901E550FC4FD5
:1039E0000491877010E0082E02C0159507950A947F
:1039F000E2F701701127F901E551FC4FE490F12C39
:103A0000082E02C0F594E7940A94E2F791E0E922C7
:103A1000FF24F901E552FC4FC491D0E002C0D595D6
:103A2000C7958A95E2F7C170DD270115110519F0D8
:103A300081EE0E94F508E114F10419F086EE0E946F
:103A4000F5088D2D0E94280AE114F10419F086EE84
:103A50000E94A4090115110519F081EE0E94A40924
:103A6000CD2B19F08CE20E94280ACDB7DEB7E7E033
:103A70000C94B62DEF92FF920F931F93CF93DF9389
:103A8000EC01162F0AE08881882309F455C08130A3
:103A900009F043C08981813041F47E0182E0E80E63
:103AA000F11C8A810E94280A09C0823049F47E01F3
:103AB000E2E0EE0EF11C8A810E94F508E7012FC0BA
:103AC000833041F47E01F2E0EF0EF11C8A810E9406
:103AD000A409F4CF843011F0219621C02A812296C6
:103AE00080E090E030E0205331092A30310558F46D
:103AF000089FA001099F500D1124C901840F951F33
:103B000021962881EFCF009751F0EFE9FFE0319740
:103B1000F1F700C000000197F6CF0E94DD1C21964E
:103B2000812F882309F4AFCFEFE9FFE03197F1F758
:103B300000C000008150F5CFCDB7DEB7E6E00C94B1
:103B4000B72D809102011F928F93809103011F92E4
:103B50008F93809106011F928F93809107011F928E
:103B60008F93809108011F928F93809109011F927A
:103B70008F938BE094E09F938F930E94C4068DB740
:103B80009EB70E960FB6F8949EBF0FBE8DBF0895D8
:103B9000883220F58E3108F068C08B3091F1C0F486
:103BA000873009F0BEC081E08093090184E18093F1
:103BB00008018AE0809307018EE18093060188E086
:103BC0008093030188E2809302018DE695E0C6C0F0
:103BD000833109F443C0843169F1A3C08F3409F4FF
:103BE0009EC028F4893231F1883359F09AC081356A
:103BF00031F008F4D4C0823509F4A7C092C08FEF29
:103C0000A5C08FE895E00E942B060E94A11D1F927F
:103C100081E08F931F9288E08F9388E894E09F93D0
:103C20008F930E94C4060F900F900F900F900F90EB
:103C30000F9096C08CE895E00E942B0680914E0371
:103C4000882309F4AAC010924E0310924D031092DB
:103C50004C0310924B0310924A03B1C08EE795E0DB
:103C60000E942B060E94A11D7BC08D5180934E03A4
:103C7000833031F170F48130D1F0823009F03FC0EF
:103C800088E091E090934D0380934C038CE991E0A0
:103C90001FC0853059F108F1863089F582E091E046
:103CA00090934D0380934C0387ED91E011C089E020
:103CB00091E090934D0380934C0383E991E008C019
:103CC00087E091E090934D0380934C0388EA91E064
:103CD00090934B0380934A0318C086E091E0909341
:103CE0004D0380934C0385EB91E0F2CF83E091E0AC
:103CF00090934D0380934C0384EC91E0E9CF1092B4
:103D00004E038BE795E00E942B0680914E0388239B
:103D100009F455C01F928F9387E795E00DC08AE0A4
:103D200015C08AE695E01AC097FF47C010828081CF
:103D30001F928F9384E695E09F938F930E94C40611
:103D40000F900F900F900F900BC081E0E0914C030B
:103D5000F0914D03309729F581E695E00E942B06FE
:103D600020914E03222359F180914A0390914B03F5
:103D7000009711F48FE891E09F938F931F922F93F8
:103D800088E595E09F938F930E94C4060F900F9053
:103D90000F900F900F900F9016C080E0089586EF5F
:103DA000D5CF2081082E000C990B820F911D8F3FDB
:103DB000910509F00CF4B8CF8FEF8083B8CF84E57C
:103DC00095E00E942B0681E00895CF93C82F1F92A3
:103DD0008F9385EA95E09F938F930E94C40681E0BC
:103DE00001C0880FCA95EAF70E94F10C0E94950C59
:103DF0000F900F900F900F90CF910895EF92FF9238
:103E00000F931F93CF93DF938B3109F4FEC008F01B
:103E10009FC08B3009F4C2C008F07DC0863009F421
:103E2000C0C020F4853009F4CEC05FC1873009F4EA
:103E3000D1C0883009F059C10E9445121F928F935A
:103E40008DE299E09F938F930E94C4060E944012D6
:103E500083FB992790F91F929F9382FB992790F9F2
:103E60001F929F9381FB992790F91F929F93982F00
:103E700091701F929F931F928F9384EE98E09F936F
